:0200000480007A
:100000006F000005732F2034930F80006308FF03F7
:10001000930F90006304FF03930FB0006300FF038E
:10002000130F000063040F0067000F00732F2034CC
:1000300063540F006F00400093E19153171F0000BD
:1000400023223FFC171F000023200FFC6FF01FFF2F
:100050009300000013010000930100001302000050
:100060009302000013030000930300001304000038
:100070009304000013050000930500001306000020
:100080009306000013070000930700001308000008
:10009000930800001309000093090000130A0000F0
:1000A000930A0000130B0000930B0000130C0000D8
:1000B000930C0000130D0000930D0000130E0000C0
:1000C000930E0000130F0000930F0000732540F102
:1000D0006310050097020000938202017390523072
:1000E000735044749702000093820201739052305F
:1000F00073500018970200009382420273905230AE
:100100009B021000939252039382F2FF7390023B82
:100110009302F0017390023A73504030970200004E
:1001200093824201739052307350203073503030BC
:100130009301000097020000938202ED7390523009
:10014000130510001315F501635C05000F00F00F97
:10015000930110009308D005130500007300000000
:1001600093020000638A020073905210B7B200003D
:100170009B829210739022307350003097020000DF
:100180009382420173901234732540F17300203042
:1001900093012000B7000080130100003BD72040EE
:1001A000B70300806314776293013000B7000080CA
:1001B000130110003BD72040B70300C063187760DD
:1001C00093014000B7000080130170003BD720402E
:1001D000B70300FF631C775E93015000B7000080F7
:1001E0001301E0003BD72040B703FEFF6310775EAA
:1001F00093016000B70000809B8010001301F001A4
:100200003BD720409303F0FF6312775C93017000AB
:10021000B70000809B80F0FF130100003BD7204017
:10022000B70300809B83F3FF6312775A930180002A
:10023000B70000809B80F0FF130110003BD72040E7
:10024000B70300409B83F3FF63127758930190003C
:10025000B70000809B80F0FF130170003BD7204067
:10026000B70300019B83F3FF631277569301A0004D
:10027000B70000809B80F0FF1301E0003BD72040D7
:10028000B70302009B83F3FF631277549301B0001E
:10029000B70000809B80F0FF1301F0013BD72040A6
:1002A00093030000631477529301C000B7808181EB
:1002B0009B801018130100003BD72040B783818139
:1002C0009B831318631477509301D000B78081810A
:1002D0009B801018130110003BD72040B7C3C0C04B
:1002E0009B83030C6314774E9301E000B7808181F8
:1002F0009B801018130170003BD72040B70303FF09
:100300009B8333306314774C9301F000B780818175
:100310009B8010181301E0003BD72040B703FEFF7D
:100320009B8363606314774A93010001B7808181E6
:100330009B8010181301F0013BD720409303F0FF7E
:100340006316774893011001B78081819B80101854
:10035000130100FE3BD72040B78381819B83131894
:100360006316774693012001B78081819B80101826
:10037000130110FE3BD72040B7C3C0C09B83030CC2
:100380006316774493013001B78081819B801018F8
:10039000130170FE3BD72040B70303FF9B8333302C
:1003A0006316774293014001B78081819B801018CA
:1003B0001301E0FE3BD72040B703FEFF9B83636041
:1003C0006316774093015001B78081819B8010189C
:1003D0001301F0FF3BD720409303F0FF6318773EF3
:1003E0009301C002B720F1FF9B8050349390C0006E
:1003F00093808067130100003BD72040B75334122D
:100400009B8383676314773C9301D002B720F1FF8D
:100410009B8050349390C00093808067130140000C
:100420003BD72040B74323019B8373566310773A31
:100430009301E002B72009009B8050349390C000E4
:1004400093808067130100003BD72040B75334925C
:100450009B838367631C77369301F002B720090002
:100460009B8050349390C0009380806713014000BC
:100470003BD72040B74323F99B83735663187734E7
:1004800093016001B700008013017000BBD02040D1
:10049000B70300FF639C703293017001B7000080C6
:1004A0001301E0003BD12040B703FEFF631071321F
:1004B0009301800193007000BBD0104093030000B3
:1004C000639670309301900113020000B700008022
:1004D000130170003BD720401303070013021200E2
:1004E00093022000E31452FEB70300FF6310732E43
:1004F0009301A00113020000B70000801301E00087
:100500003BD7204013000000130307001302120022
:1005100093022000E31252FEB703FEFF6318732A12
:100520009301B00113020000B70000801301F00135
:100530003BD7204013000000130000001303070006
:100540001302120093022000E31052FE9303F0FF07
:10055000631E73269301C00113020000B7000080E0
:10056000130170003BD720401302120093022000B9
:10057000E31652FEB70300FF631A77249301D001FC
:1005800013020000B70000801301E0001300000018
:100590003BD720401302120093022000E31452FEC6
:1005A000B703FEFF631477229301E00113020000FA
:1005B000B70000801301F0011300000013000000D9
:1005C0003BD720401302120093022000E31252FE98
:1005D0009303F0FF631C771E9301F00113020000E8
:1005E000B700008013000000130170003BD72040CB
:1005F0001302120093022000E31452FEB70300FF1F
:100600006316771C9301000213020000B7000080FC
:10061000130000001301E000130000003BD720404E
:100620001302120093022000E31252FEB703FEFFF2
:10063000631E77189301100213020000B7000080B8
:1006400013000000130000001301F0013BD720400D
:100650001302120093022000E31252FE9303F0FFF4
:100660006316771693012002130200001301700035
:10067000B70000803BD720401302120093022000F5
:10068000E31652FEB70300FF6312771493013002A2
:10069000130200001301E000B70000801300000007
:1006A0003BD720401302120093022000E31452FEB5
:1006B000B703FEFF631C7710930140021302000092
:1006C0001301F001B70000801300000013000000C8
:1006D0003BD720401302120093022000E31252FE87
:1006E0009303F0FF6314770E93015002130200008E
:1006F0001301700013000000B70000803BD72040BA
:100700001302120093022000E31452FEB70300FF0D
:10071000631E770A93016002130200001301E000D8
:1007200013000000B7000080130000003BD72040FA
:100730001302120093022000E31252FEB703FEFFE1
:100740006316770893017002130200001301F00191
:100750001300000013000000B70000803BD72040CA
:100760001302120093022000E31252FE9303F0FFE3
:10077000631E7704930180029300F0003B51104008
:10078000930300006314710493019002930000022C
:100790003BD1004093030002631A71029301A0024F
:1007A000BB50004093030000639270029301B002BB
:1007B00093000040371100001B0101803BD0204016
:1007C0009303000063147000631030020F00F00FF9
:1007D000638001009391110093E111009308D0050B
:1007E00013850100730000000F00F00F930110004B
:1007F0009308D0051305000073000000731000C0BB
:1008000000000000000000000000000000000000E8
:1008100000000000000000000000000000000000D8
:1008200000000000000000000000000000000000C8
:0C083000000000000000000000000000BC
:1010000000000000000000000000000000000000E0
:1010100000000000000000000000000000000000D0
:1010200000000000000000000000000000000000C0
:1010300000000000000000000000000000000000B0
:081040000000000000000000A8
:040000058000000077
:00000001FF
